:020000040000FA
:0600000025006800870ADC
:10001000560831082E083308200877087708770833
:100020002E086E0869086B0861086D0865086C0881
:1000300065086308740872086F086E086908630829
:1000400073082E0863086F082E0875086B080F0EDA
:10005000E201300831083208330834083508360820
:100060003708380839084108420843084408450859
:100070004608E2015408650873087408200824083B
:10008000FF082A000000EA02430A0008410C2A0087
:100090004B0A890C2A00EA024B0A300829000002A8
:1000A0002D00A40200022E00A40200022F00A402D0
:1000B00000023000A40200023100A402000232005B
:1000C000A40200023300A40200023400A4020002D1
:1000D0003500B30C7503740373037203710370036B
:1000E0006F036E036D030306AD01E9026A0A30086F
:1000F000080C2900260549092B03030726050306DA
:1001000026044909E9027C0A260449090008090C69
:1001100024006000A4028407890AC70C02002C0C8A
:10012000060026006607F70A170C24006C00080C6E
:100130002900A606B00A4606990A6C000C02390985
:100140002000FF0F4306A70AA402AC029E0A880300
:1001500027092000A402080227092000A802C00ADB
:10016000460949090304A60703052B03E902B10A5E
:10017000460949090B022000A402AC026C07970A49
:10018000860500007F00170C2400400C4E090D026C
:100190003F000605580C2900000C3500090C3600FC
:1001A0007F037E037D037C037B037A03790378035B
:1001B0007703760375030306E20A26043D0C410922
:1001C0002605E70A26053D0C4109260400003D0CE2
:1001D0004109E902D00A660000004606870A150CAC
:1001E00029006100E107F20AE902F10A870A010C1D
:1001F0002600180C240084024306180C240000007A
:10020000000000000000000000000304A606030533
:100210006003960C80014306120B00000000040CE2
:100220002C00FB0A00000000EC02FB0A8605860495
:10023000480C29003C0C4109860586040304A606E7
:1002400003057F037E037D037C037B037A0379032D
:1002500078037703A6072F0BA6062C0B310BA607F6
:100260002F0B5A0C4109E9021C0B170C2400400CFF
:100270004E092D024307870A0604170C240046077F
:100280003F0B61004107420B00022B00780961001F
:100290004107480BA402AC026C073F0B0605870A16
:021FFE00E20FF0
:00000001FF
